:100000000C9417060C946C290C9499290C943F06B7
:100010000C943F060C943F060C943F060C943F064C
:100020000C943F060C943F060C94BF0C0C943F06B6
:100030000C943F060C943F060C943F060C943F062C
:100040000C94C6290C943F060C94802D0C94BB2D67
:100050000C943F060C943F060C943F060C943F060C
:100060000C943F060C943F06921C991C991C921C00
:10007000991C991C991C991C991C991C991C991CD8
:10008000991C991C991C991C991C071C991C991C5A
:10009000991C991C991C711B991C991C991C991CE1
:1000A000991C991C991C991C991C991C991C991CA8
:1000B000991C991C991C131C131C131C131C131C36
:1000C000131C131C131C131C991C991C991C991CA0
:1000D000991C991C711B121C121C121C121C991CBD
:1000E000231C2B1C331C3B1C431C4B1C531C5B1C38
:1000F000651C6F1C791C831CB61B761B991C991CF4
:10010000991C991C071C991C991C991C991C991CD9
:10011000991C991C991C111C111C111C111C991C57
:10012000231C2B1C331C3B1C431C4B1C531C5B1CF7
:10013000651C6F1C791C831CB61B761B991C991CB3
:10014000991C991C071CCA1CCA1CCA1CCA1CCA1CA4
:10015000CA1CCA1CCA1CCA1CCA1CCA1CCA1CCA1C6F
:10016000EA1DEA1DEA1DEA1DEA1DEA1D111D1B1DFF
:10017000251D2F1D951D9F1DAD1DBE1D5B1ECB1E7C
:100180009C1EA11EA61EAB1EB01EB51EBA1ECB1E07
:10019000C51EE425F92505260E261B2641264926DF
:1001A0006C265926456E746572206D656E752E2E0F
:1001B0002E00546F67676C6564206D6963726F50C1
:1001C000504D00546F67676C656420696E76657288
:1001D0007465642050504D2100546F67676C6564EE
:1001E000205458206D7574696E672100546F6767DD
:1001F0006C65642074656C656D657472792100505E
:10020000726F746F636F6C206572726F72207769A2
:1002100074682052580054696D656F757420776852
:10022000656E20636F6E6E656374696E6720746FB0
:1002300020525800507265737320616E79206B658F
:100240007920746F2063616E63656C00436F6E6E1E
:10025000656374696E6720746F2052582C20706F2C
:100260007765722075702074686520525820287751
:100270006974682062696E6420706C7567206966B5
:10028000206E6F74207573696E6720616C77617979
:10029000732062696E642900546F67676C6564201F
:1002A00027696D6D656469617465206F757470751B
:1002B000742700546F67676C65642027736C6176E0
:1002C00065206D6F64652700546F67676C656420F7
:1002D00027616C776179732062696E642700546FBF
:1002E00067676C65642050504D206368616E6E6571
:1002F0006C206C696D6974005365742052535349C6
:1003000020696E6A656374696F6E206368616E6EE2
:10031000656C2028303D3D64697361626C6529001D
:100320005365742050504D206D696E696D756D2058
:1003300073796E630053657420626561636F6E202C
:10034000696E74657276616C0053657420626561D4
:10035000636F6E2064656C6179005365742062651B
:1003600061636F6E206672657175656E6379206971
:100370006E20487A3A20303D64697361626C652C66
:100380002050783D504D52206368616E6E656C2040
:10039000782C2046783D465253206368616E6E6526
:1003A0006C2078005365742050574D2073746F7023
:1003B0002064656C61792028302064697361626C07
:1003C00065642C20312D323535203D3D20302E31D5
:1003D00073202D2035306D696E29005365742050CF
:1003E000504D2073746F702064656C6179202830E3
:1003F0002064697361626C65642C20312D3235355F
:10040000203D3D20302E3173202D2035306D696E1A
:100410002900536574206661696C736166652064A8
:10042000656C61792028302064697361626C656451
:100430002C20312D323535203D3D20302E3173209A
:100440002D2035306D696E29002A2A2A2A2A2A2A67
:100450002A2A2A2A2A2A2A2A2A2A2A2A2A2A2A2AFC
:100460002A2A2A2A2A2A0052582041636B656420CE
:100470002D2072657665727420737563636573737E
:1004800066756C21002A2A2A2A2A2A2A2A2A2A2A36
:100490002A2A2A2A2A2A2A2A2A2A2A2A2A2A2A2ABC
:1004A0002A2A002A2A2A2A2A2A2A2A2A2A2A2A2AD6
:1004B0002A2A2A2A2A2A2A2A2A2A2A2A2A2A2A2A9C
:1004C0000052582041636B6564202D207570646173
:1004D0007465207375636365737366756C21002A98
:1004E0002A2A2A2A2A2A2A2A2A2A2A2A2A2A2A2A6C
:1004F0002A2A2A2A2A2A2A2A2A2A2A2A0056616CE1
:1005000069642063686F69636573206172653A206E
:100510005B315D2D5B31365D20286368616E6E65F1
:100520006C20312D31362900536574206F7574703D
:10053000757420666F7220706F727420005B585D56
:100540002061626F7274206368616E6765732061F9
:100550006E64206578697420525820636F6E6669F6
:1005600067005B535D207361766520736574746901
:100570006E677320746F205258005B525D20726565
:10058000766572742052582073657474696E67734F
:1005900020746F2064656661756C747300557365B3
:1005A000206E756D62657273205B312D445D207421
:1005B0006F206564697420706F727473205B452DC1
:1005C000515D20666F722073657474696E67730085
:1005D000202D20726563656976657220636F6E6693
:1005E0006967757261746F722C207278207377203E
:1005F000000A0A6F70656E4C52536E672000536597
:10060000742073657269616C2062617564726174D3
:10061000653A200056616C69642063686F696365A0
:10062000733A2031202D20342B34202F2032202DDE
:100630002038202F2033202D20382B34202F203419
:10064000202D203132202F2035202D2031322B3407
:10065000202F2036202D203136005365742043682A
:10066000616E6E656C20636F6E6669673A20005339
:1006700065742044617461726174652028302D3284
:10068000293A200053657420486F70206368616EBA
:100690006E656C7320286D61782032342C20736570
:1006A0007061726174656420627920636F6D6D6141
:1006B00073292076616C69642076616C756573209E
:1006C000312D3235353A2000536574206368616EF0
:1006D0006E656C2073706163696E672028783130B5
:1006E0006B487A293A200053657420524620706F77
:1006F0007765722028302D37293A20005365742001
:100700005246206D616769632028686578292065F5
:100710002E672E20307844454144463030443A20FC
:10072000005365742062617365206672657175653A
:100730006E63792028696E20487A293A20005B5A36
:100740005D20656E74657220726563656976657299
:1007500020636F6E66696775726174696F6E20756C
:1007600074696C79005B465D20646973706C6179B3
:100770002061637475616C206672657175656E6366
:100780006965732075736564005B525D2063616CFD
:1007900063756C6174652072616E646F6D206B654A
:1007A0007920616E6420686F70206C697374005BDF
:1007B000495D207265696E697469616C697A65204A
:1007C00073657474696E677320746F20736B6574DE
:1007D00063682064656661756C7473005B585D20A6
:1007E000726576657274206368616E6765732061F7
:1007F0006E642065786974206D656E75005B535D6D
:1008000020736176652073657474696E67732074F4
:100810006F20454550524F4D20616E6420657869C8
:1008200074206D656E7500557365206E756D62651B
:100830007273205B302D395D20746F20656469749C
:1008400020706172616D657465727300202D205394
:10085000797374656D20636F6E6669677572617414
:10086000696F6E000A0A6F70656E4C52536E672096
:10087000005129204F7574707574206265666F721F
:1008800065206C696E6B20283D465329203A200074
:10089000502920536C617665206D6F646520286552
:1008A00078706572696D656E74616C293A20004FCD
:1008B000292054696D65642042494E4420617420AA
:1008C0007374617274757020203A20004E29205094
:1008D000504D206F7574707574206C696D69746506
:1008E0006420202020203A200044495341424C45B6
:1008F00044004D292050504D205253534920746FCD
:10090000206368616E6E656C202020203A20004CC8
:10091000292050504D206D696E696D756D20737979
:100920006E63202875732920203A200044495341E2
:10093000424C4544004B29204661696C73616665F1
:1009400020626561636F6E20696E74762E20283197
:100950002D32353573293A20004A29204661696CC9
:100960007361666520626561636F6E2064656C61AA
:10097000792028302D323535203D3E20313073200E
:100980002D203135306D696E293A200049292046E5
:1009900061696C7361666520626561636F6E206674
:1009A00072712E203A200048292050574D20737430
:1009B0006F702064656C6179202020202020203A0F
:1009C000200047292050504D2073746F70206465BB
:1009D0006C6179202020202020203A200046292008
:1009E0004661696C736166652064656C617920207D
:1009F00020202020203A200050574D206368616E4F
:100A00006E656C200066756E6374696F6E3A2000C7
:100A10002920706F72742000506F776572546F7761
:100A2000657200445446205548462033322D626991
:100A3000742031306368004F70656E4C52536E679E
:100A40005258206D696E6920342F36636800466CF9
:100A50007974726F6E2F4F72616E676552582055B0
:100A600048462038636800525820747970653A20EF
:100A70000044697361626C656400487A00203D3D02
:100A8000200043616C63756C617465642070616300
:100A90006B657420696E74657276616C3A200042F1
:100AA00029204D6963726F202868616C6629205087
:100AB000504D202020203A00412920496E76657251
:100AC0007465642050504D20696E20202020203A0B
:100AD000003029204D7574652062757A7A65722020
:100AE000286D6F73746C79293A0039292053657227
:100AF00069616C2062617564726174653A00736D3E
:100B0000617274506F7274004672536B7900547244
:100B1000616E73706172656E740044697361626CBA
:100B200065640038292054656C656D657472793A86
:100B300020202020202020003729204368616E6E6D
:100B4000656C20636F6E6669673A20200036292045
:100B500044617461726174652028302D32293A2015
:100B6000202000352920486F70206368616E6E6513
:100B70006C733A2020202020003429204368616EC5
:100B80006E656C2073706163696E673A2020003374
:100B90002920524620706F7765722028302D372922
:100BA0003A202020003229205246206D6167696377
:100BB0003A202020202020202020003129204261BE
:100BC0007365206672657175656E63793A202020C1
:100BD0000000000000240027002A0000000000257B
:100BE0000028002B0000000000230026002900043C
:100BF00004040404040404020202020202030303C4
:100C000003030301020408102040800102040810BD
:100C1000200102040810200000000700020100006B
:100C2000030406000000000000000000632F1124F0
:100C30001FBECFEFD8E0DEBFCDBF13E0A0E0B1E034
:100C4000E8E0F1E602C005900D92A839B107D9F7A6
:100C500016E0A8E9B3E001C01D92AD35B107E1F798
:100C60001CE0CEE2DCE004C02297FE010E945F306F
:100C7000CC32D107C9F70E94A82F0C9482300C9473
:100C80000000A0E0B0E0E7E4F6E00C942E30EC01C8
:100C9000A880B980CA80DB80A114B104C104D1044A
:100CA00041F484E2A82E89EDB82E8BE5C82E87E0AA
:100CB000D82EC601B5012DE133EF41E050E00E948E
:100CC0000B3027EA31E440E050E00E94B72F7B016F
:100CD0008C01C601B5012DE133EF41E050E00E94E7
:100CE0000B30CA01B9012CEE34EF4FEF5FEF0E94D9
:100CF000B72F6E0D7F1D801F911F97FF04C061509D
:100D0000704080409048688379838A839B839B01ED
:100D1000AC015F77B901CA01CDB7DEB7EAE00C9448
:100D20004A300E944106089581EB92E00E944106FC
:100D300008956093B1027093B2028093B3029093CE
:100D4000B4020895A0E0B0E0E8EAF6E00C942730A1
:100D5000EC012B016A016115710519F0FB0191830A
:100D60008083C114D10449F0C6010297839728F00B
:100D700020E030E040E050E0DCC0A9908A2D90E017
:100D80000E947730892BC9F7FDE2AF1621F4A990B4
:100D90003324339405C08BE2A81609F4A9903324B8
:100DA000C114D10421F0E0E1CE16D10411F5F0E335
:100DB000AF1669F48881883711F0883541F4A9802D
:100DC000229682E0382A20E1C22ED12C12C0C11412
:100DD000D10479F4E0E3AE1659F199E9E92E99E9E5
:100DE000F92E99E9092F99E1192F8AE0C82ED12C03
:100DF0003AC0FAE0CF16D10491F080E1C816D104D0
:100E000029F0E8E0CE16D104F9F415C0BFEFEB2EBF
:100E1000BFEFFB2EBFEF0B2FBFE01B2F24C0A9E9B4
:100E2000EA2EA9E9FA2EA9E90A2FA9E11A2F1BC077
:100E3000F8E0CF2ED12CEFEFEE2EEFEFFE2EEFEFFE
:100E40000E2FEFE11E2F0FC09601442737FD40956E
:100E5000542F6FEF7FEF8FEF9FEF0E94E92FC901B3
:100E6000DA017C018D0120E030E040E050E060E0FC
:100E70003601882477FC8094982C70EDB72EBA0C3C
:100E8000F9E0FB1570F48A2D81548A3118F499EC3D
:100E9000B92E06C08A2D81568A3148F589EAB82EC6
:100EA000BA0C8B2D90E08C159D050CF56F3FE9F089
:100EB000E216F30604071507B8F0CA01B901A40148
:100EC00093010E94B72F9B01AC018B2D90E0A0E015
:100ED000B0E0280F391F4A1F5B1F281739074A0740
:100EE0005B0710F061E001C06FEFA990C6CF41141D
:100EF000510451F0662311F0219703C031FE04C064
:100F00002297F201D183C08330FE07C050954095EF
:100F1000309521953F4F4F4F5F4F67FF0AC082E2E8
:100F200090E090935C0680935B062FEF3FEF4FEFCE
:100F30005FEFB901CA01CDB7DEB7E1E10C944330F0
:100F4000FC0188279927E89421912032E9F3293080
:100F500010F02E30C8F32B3241F02D3239F4689462
:100F600004C00E94F507820F911D219120532A3061
:100F7000C0F31EF4909581959F4F089548E953E082
:100F80000E94C3070895009731F4DA018D919C9176
:100F9000009709F40EC0DC01FB013D912191222351
:100FA00019F03217C9F3FACF332331F4DA011D9265
:100FB0001C928827992708951197AF93BF93FB013F
:100FC0003D912191321771F4332321F48827992719
:100FD000119702C01E921196FA01A193B0839F91BE
:100FE0008F910895222369F7EACF7AE0979F902D99
:100FF000879F802D910D1124089580919A0381304F
:1010000019F482E080939A0380919A03833019F453
:1010100084E080939A030895E3E0F0E089E0809310
:101020005700849190E08670863009F491E0892F12
:1010300008951F93182F0E940C08882379F09FB7FA
:1010400081E08093A305F894A89588E180936000DF
:1010500010936000112309F0A8959FBF1F91089578
:10106000382F20E08091350590913605822793270F
:1010700040E061E270E19C01220F331F97FF04C042
:10108000C9018627972701C0C9014F5F483099F7EA
:101090009093360580933505089587E38093D003B8
:1010A00080E092ECA1E0B0E08093D1039093D20372
:1010B000A093D303B093D40387E08093DD0380E053
:1010C00091EAACEBB3E38093D5039093D603A0935E
:1010D000D703B093D80385E08093DE038DEE9EEFB7
:1010E000ADEABEED8093D9039093DA03A093DB03BE
:1010F000B093DC03AFEDB3E080E090E0863010F019
:10110000E0E004C0FC01EF57FC4FE081ED93019655
:101110008831910599F782E08093F7038AE0809304
:10112000F803089580E09EECADEEB4E380939D0358
:1011300090939E03A0939F03B093A00380E090E060
:10114000A0E0B0E58093A1039093A203A093A30332
:10115000B093A403E5EAF3E080E081938F5F8031F0
:10116000E1F708958436910520F4BC0180E090E019
:1011700025C08E3B910550F48A559040BC0180E01B
:1011800090E02AE030E040E050E016C0823D91055A
:1011900050F4845B9040BC0180E090E024E630E0B5
:1011A00040E050E009C08D5C9040BC0180E090E0E0
:1011B00028E532E040E050E00E94B72F24E630E01E
:1011C00040E050E00E94B72F089590E08C599F4F67
:1011D0000E94B2080895DC019896EC91F0E0E77067
:1011E000F070E758FC4F808108958F929F92AF92E4
:1011F000BF92CF92DF92EF92FF920F931F938C01D9
:101200000E94EB08D80197962C9130E043E150E022
:10121000249FF001259FF00D349FF00D1124EB5415
:10122000FD4F80809180A280B38090E00F96AA2726
:1012300097FDA095BA2FBC01CD0120E43FE14DE719
:1012400050E00E94B72FA50194010E94E92F690187
:101250007A0180ED97E0A0E0B0E0C80ED91EEA1E4A
:10126000FB1ED80198968C91887181F060E07EEE2B
:101270008AEB9BE0A50194010E94E92F28513C4F85
:101280004F4F5F4FC20ED31EE41EF51E87EE93E054
:10129000A0E0B0E0C80ED91EEA1EFB1EC701B601D1
:1012A00028EE33E040E050E00E94E92FCA01B90186
:1012B00028EE33E040E050E00E94B72F1F910F91DD
:1012C000FF90EF90DF90CF90BF90AF909F908F9066
:1012D00008958F3F910509F010F480E0089522E011
:1012E0008030920710F481E008958050934010F010
:1012F00083E0089582E00895CF92DF92FF920F93EA
:101300001F93CF93DF93F82FEB016A01182F1695E7
:10131000E0E088819981D6018C938A819B81119626
:101320008C9311978C819D8112968C9312978E814C
:101330009F8113968C931397288139814A815B8111
:101340006C817D818E819F819295990F990F907C00
:10135000832F8370982B852F8370880F880F982B8D
:10136000872F83708295807F982B14969C9385E0BD
:1013700090E0C80ED91E2896EF5F1E1750F6F0FFBA
:1013800021C0888199810E946909F82E8A819B81F8
:101390000E946909182F8C819D810E946909082F7C
:1013A0008E819F810E946909F294FF0CFF0C70EC02
:1013B000F7221295107F1F29182B000F000F012B09
:1013C000D6010C93DF91CF911F910F91FF90DF9089
:1013D000CF90089523E08032920718F420E030E0A7
:1013E00026C023E0883E920748F49C012F513340E9
:1013F00054E0369527955A95E1F719C027E0803DCE
:10140000920720F49C012C5D334011C028E08839FC
:10141000920718F02FEF33E00AC09C01285C374098
:1014200044E0369527954A95E1F72D503C4FC90188
:1014300008958C30910548F49C0174E0220F331F0D
:101440007A95E1F7285D3C4F17C023E0843F92076F
:1014500020F49C0124523C4F0FC024E080309207BE
:1014600018F020E938E008C09C012657334F64E0AB
:10147000220F331F6A95E1F7C90108959C01369543
:10148000279525753575821B930B9C0136952795FD
:10149000369527952373337383739373280F391FFE
:1014A000C901E4E096958795EA95E1F7820F931FCD
:1014B0008F709F7021E031E0AC01429FC001439FDB
:1014C000900D529F900D1124892F0895882339F093
:1014D00042980000419A0000429A00000895429804
:1014E000000041980000429A00000895429A0000CE
:1014F00086B142980000817008950F931F93082FC2
:101500005C9A42985C9810E0802F80780E94660A6E
:10151000000F1F5F1830C1F742981F910F91089577
:101520008F770E947D0A08950F931F93082F10E074
:10153000802F80780E94660A000F1F5F1830C1F765
:1015400042981F910F9108950F931F93429880E046
:1015500000E0182F110F0E94760A810F0F5F0830EC
:10156000C1F71F910F9108950E94900A0E94A40A4A
:101570005C9A08951F93162F80680E947D0A812F20
:101580000E94940A5C9A1F9108951F931091D903A9
:101590001827E0EDF3E0E80FF11D89E767850E9469
:1015A000BA0A8DE3612F0E94BA0A82E4612F0E9479
:1015B000BA0A1F91089586E20E94B40A08950F9313
:1015C0001F938C018CE1F80164810E94BA0A8DE1BD
:1015D000F80165810E94BA0A8EE1F80166810E94D5
:1015E000BA0A80E2F80167810E94BA0A81E2F80132
:1015F00060850E94BA0A82E2F80161850E94BA0AF7
:1016000083E2F80162850E94BA0A84E2F8016385E8
:101610000E94BA0A85E2F80164850E94BA0A8AE249
:10162000F80165850E94BA0A8EE6F80166850E9477
:10163000BA0A8FE6F80167850E94BA0A80E7F801C6
:1016400060890E94BA0A81E7F80161890E94BA0A9A
:1016500082E7F80162890E94BA0A1F910F910895EA
:10166000EF92FF920F931F93CF93DF937B018C0137
:10167000603028E372072CE982072CE1920728F5F5
:1016800020E836E948E950E00E94E92FE90168972F
:10169000B90180E090E020E839E647E65FEF0E947C
:1016A000B72F6E0D7F1D801F911F22E0660F771FE1
:1016B000881F991F2A95D1F721E732E040E050E0DA
:1016C0000E94E92F890180E421C020E03DE241E34E
:1016D00051E00E94E92FE9016897B90180E090E0AC
:1016E00020E033ED4EEC5EEF0E94B72F6E0D7F1DB4
:1016F000801F911F660F771F881F991F21E732E017
:1017000040E050E00E94E92F890180E69E012F71A0
:10171000622F680F85E70E94BA0A86E7612F0E9450
:10172000BA0A87E7602F0E94BA0ACDB7DEB7E6E0B3
:101730000C944E30682F8DE60E94BA0A08959F924D
:10174000AF92BF92CF92DF920F93DF93CF9300D0EF
:1017500000D0CDB7DEB7982E83E00E94B40A809304
:10176000F90384E00E94B40A8093FA0386E060E003
:101770000E94BA0A87E061E00E94BA0A89E06FE736
:101780000E94BA0A8AE065E00E94BA0A8BE062E130
:101790000E94BA0A8CE065E10E94BA0A8DE06DEF02
:1017A0000E94BA0A8EE060E00E94BA0A992019F0FD
:1017B00084E193E008C08091F70323E1829FC00198
:1017C00011248B549D4F0E94DF0A80E36CE80E9435
:1017D000BA0A82E36FE00E94BA0A83E362E40E94DD
:1017E000BA0A84E36AE00E94BA0A85E36AE20E94C8
:1017F000BA0A86E36DE20E94BA0A87E364ED0E94AA
:10180000BA0A88E360E00E94BA0A89E360E00E94B5
:10181000BA0A992049F055E8A52E51ECB52E51ECA5
:10182000C52E5EEDD52E08C0A090D903B090DA0386
:10183000C090DB03D090DC030AE38D2D9927AA2703
:10184000BB2789839A83AB83BC83802F69810E94E5
:10185000BA0A802F8B5F69810E94BA0ADC2CCB2CDC
:10186000BA2CAA240F5F0E3341F783E46FEF0E9476
:10187000BA0A84E46FEF0E94BA0A85E46FEF0E940F
:10188000BA0A86E46FEF0E94BA0A992019F08DE631
:1018900066E003C08DE66091DD030E94BA0A89E725
:1018A00060E00E94BA0A8AE76091DE030E94BA0AE9
:1018B00083E760E00E94BA0A84E760E00E94BA0A07
:1018C000992029F060E071EA8CEB93E308C0609105
:1018D000D5037091D6038091D7039091D8030E94CD
:1018E000300B0F900F900F900F90CF91DF910F91D1
:1018F000DF90CF90BF90AF909F90089587E061E018
:101900000E94BA0A8EE764E20E94BA0A88E063E0A5
:101910000E94BA0A88E060E00E94BA0A87E065E0A7
:101920000E94BA0A85E062E00E94BA0A83E00E943F
:10193000B40A8093F90384E00E94B40A8093FA0306
:101940000895582F40919E04842F90E0FC01EF7081
:10195000F0709F012F5F3F4F64E0959587956A95E2
:10196000E1F72817390751F0E257FB4F5083842FD6
:101970008F5F8F70407F842B80939E0408951F9209
:101980000F920FB60F9211241F932F933F934F93F3
:101990005F936F937F938F939F93AF93BF93CF93F7
:1019A000DF93EF93FF93C0918600D0918700209141
:1019B000E2043091E3048091C104882309F062C0FD
:1019C000BE01621B730B2091A1033091A2034091D1
:1019D000A3035091A40325FD02C07695679589E085
:1019E000653C7807B8F180914703BCE1569547956F
:1019F00037952795BA95D1F7211531054105510540
:101A000021F421E030E040E050E090E0A0E0B0E0E0
:101A1000281739074A075B07D0F4809147038F3FA7
:101A2000B1F020E00EC0E22FF0E0EE0FFF1FDF016B
:101A3000AE53BB4F8D919C91E95DFC4F91838083A8
:101A40002F5F80914703281770F31092C004109203
:101A5000470318C082E06D3B780760F1809147032F
:101A6000803140F510914703CB010E94EA09E12F34
:101A7000F0E0EE0FFF1FEE53FB4F918380831F5F5B
:101A800010934703D093E304C093E204FF91EF91D6
:101A9000DF91CF91BF91AF919F918F917F916F9186
:101AA0005F914F913F912F911F910F900FBE0F901B
:101AB0001F9018958FEF80934703E4CF83E08093C6
:101AC00080008AE9809381008091A10386FD05C092
:101AD000809181008064809381008FEF9FEF9093CD
:101AE00089008093880080916F00806280936F00EE
:101AF00008956F3018F086958058089589E0689FA2
:101B0000802D11240895882319F460E071E002C04B
:101B100063E071E089E396E00E946B2D0895A0E0F8
:101B2000B0E0E5E9FDE00C943030182F0E941C2A4B
:101B30009B01AC0180912F0590913005A09131055A
:101B4000B091320569017A01C81AD90AEA0AFB0A7A
:101B5000D701C60189589341A040B04010F01092BF
:101B60002E0520932F053093300540933105509377
:101B700032052091C104822F81508230E8F5809196
:101B80002E05882309F44FC1813011F482E0BCC1D5
:101B9000803108F035C1E82FF0E0EE53FB4F1083A1
:101BA0008F5F80932E05803109F0B0C1A4ECB4E0C2
:101BB000213039F41196EC911197E695E6958C91C8
:101BC00009C08D919C911197E92FE695E695E695D0
:101BD00096958795E03140F4F0E090E0EE0FFF1F1E
:101BE000E95DFC4F918380831092C004129684E0DB
:101BF000A23DB807E9F68AC1233009F004C18091FB
:101C00002E05882321F41F3009F080C10CC18831D2
:101C100030F4E82FF0E0EF53FB4F108374C18831AC
:101C200009F0EEC0112309F0EBC0C0E0D0E00BE0FA
:101C300010E0DE0163E0AA0FBB1F6A95E1F7C09FC9
:101C4000B001C19F700DD09F700D1124FB01EE53A8
:101C5000FB4F80812181922F977095958795FD018B
:101C6000EE0FFF1FE95DFC4F91838083FB01ED5375
:101C7000FB4F30813695369536952181422F42951E
:101C8000440F407E842F832B269526952695922FF0
:101C9000977095958795FD01EE0FFF1FE75DFC4F4F
:101CA00091838083FB01EC53FB4F80818295869565
:101CB000869583704181942F990F990F292F282B96
:101CC000429546954695437082818170880F880FB2
:101CD000382F342B35952795FD01EE0FFF1FE55D5D
:101CE000FC4F31832083FB01EA53FB4F3081369553
:101CF0002181422F479544274795842F832B269592
:101D0000922F977095958795FD01EE0FFF1FE35D6C
:101D1000FC4F91838083FB01E953FB4F3081329567
:101D20003F702181422F4295407F842F832B229543
:101D30002F70922F977095958795FD01EE0FFF1FDD
:101D4000E15DFC4F91838083FB01E853FB4F808171
:101D5000881F8827881F4181942F990F292F282BAE
:101D6000441F4427441F82818370880F382F342BEF
:101D700035952795FD01EE0FFF1FEF5CFC4F31837A
:101D80002083FB01E653FB4F308136953695218148
:101D9000422F4295440F440F407C842F832B26957D
:101DA0002695922F977095958795AA0FBB1FFD01D9
:101DB000ED5CFC4F9183808365537B4FFB01208159
:101DC0002295269527704181342F330F330F330F1F
:101DD000832F822B942F9295969597709595879542
:101DE000AB5CBC4F11969C938E932196C230D1056B
:101DF00009F01FCF8091D80483FD02C01092C00467
:101E000010922E0583C0243009F080C040912E0529
:101E1000442359F4183AB1F410923605109235055E
:101E200088EA0E94300881E06FC0413019F41093B5
:101E3000330504C0423031F410933405812F0E94E1
:101E400030085DC060913405262F30E0220F331F2B
:101E5000E42FF0E0C90102968E179F0734F0433259
:101E600068F7E154FB4F1083E9CF2D5F3F4F40915E
:101E7000350550913605E217F30749F4912F80E0BC
:101E800048275927509336054093350538C0812F90
:101E900090E04817590789F580913305813069F53D
:101EA000613118F080E180933405D090340542EC24
:101EB000E42E44E0F42E00E010E01BC0F701D081D6
:101EC000C0E0818190E08C2B9D2B33E09695879527
:101ED0003A95E1F70E94EA09F801EE0FFF1FE95D6C
:101EE000FC4F918380830F5F1F4F82E090E0E80EEC
:101EF000F91E0D1518F31092C00410922E05809152
:101F00002E05882319F08F5F80932E05CDB7DEB79D
:101F1000E8E00C944C30FF920F931F93CF93DF9324
:101F2000182F092FF62E8EE30E94BA0A212F302F88
:101F3000C901EC0110E005C08FE769910E94BA0A5F
:101F40001F5F1F15C8F385E064E00E94BA0A83E0B2
:101F50000E94B40A8093F90384E00E94B40A80933B
:101F6000FA030E941C2A6093FB037093FC03809386
:101F7000FD039093FE0387E069E00E94BA0A81E0C6
:101F800080939A03CDB7DEB7E5E00C944F300E9402
:101F90008B0F80919A038130D9F40E941C2A2091E2
:101FA000FB033091FC034091FD035091FE03621B43
:101FB000730B840B950B605A76488140904040F437
:101FC000E8CF89E396E067E071E00E946B2D089509
:101FD00080919A038130A9F3089589E396E06EE732
:101FE0000E94232F0895A0E0B0E0E9EFFFE00C94F9
:101FF0002F306C0189E396E06EE70E94232F760173
:1020000000E010E0C0E0D0E0B0E2BB2E0AC0083033
:10201000110521F49E012095F60120870894E11C0A
:10202000F11CF7016081862F8D57823040F489E3DF
:1020300096E06DE70E94232FF70160816B2589E30D
:1020400096E00E94232F0115110551F0F7018081C0
:102050009E01280F311DC32FDD27C20FD31FD07063
:102060000F5F1F4F0930110591F6CDB7DEB7E9E0DC
:102070000C944B30A9E0B0E0E0E4F0E10C94363091
:10208000382FE62F8091A30490E0019664E270E07F
:102090000E94D62F982F8093A30488E9898380E13A
:1020A0008A83913071F0913028F0923099F093301A
:1020B000E1F416C085E08B8381EF8C832F5F2D8345
:1020C00017C09B8381EF8C8384E6489FC001112455
:1020D0009D830EC084E08B8381EF8C833D8308C099
:1020E0009B8381EF8C83ED8303C00E94ED0F04C0BE
:1020F000CE0101960E94F30F2996E2E00C94523033
:102100000F931F93CF93DF93182F092F89E396E046
:102110006EE70E94232F212F302FC901EC0110E020
:1021200000E288818D57823040F489E396E06DE7C4
:102130000E94232F88818027888389E396E0699114
:102140000E94232F1F5F193061F789E396E06EE745
:102150000E94232FDF91CF911F910F910895A9E045
:10216000B0E0E5EBF0E10C943630382F8091A30419
:10217000882379F48EEF89833A836B83842F90E0F0
:10218000959587958C832D83198618861F821E82CC
:102190002FC040919E04842F90E09C012F703070DE
:1021A00054E0959587955A95E1F78217930721F1A9
:1021B0008DEF89831A821B82DE01149620E008C00D
:1021C000E257FB4F80818D93405F2F5F263069F08F
:1021D000842F90E0FC0134E0F595E7953A95E1F71E
:1021E0008F709070E817F90759F740939E042A837F
:1021F000CE0101960E9480108091A30490E0019688
:1022000066E070E00E94D62F8093A3042996E2E056
:102210000C9452309F92AF92BF92CF92DF92EF9286
:10222000FF920F931F93B82EA62ED42EC22E902E5F
:102230000E941C2A7B018C0180918D0420919F04B7
:102240003091A0044091A1045091A2048823B1F0E0
:10225000D801C701821B930BA40BB50B815E9E4274
:10226000A040B04020F12C2DDC1408F42D2D8B2D36
:102270006A2D422F292D0E943A1011C0D801C701A2
:10228000821B930BA40BB50B81539547A040B04024
:1022900070F08B2D6A2D4D2D2C2D0E94AF10E092E9
:1022A0009F04F092A0040093A1041093A2041F9134
:1022B0000F91FF90EF90DF90CF90BF90AF909F90E5
:1022C000089589E396E0609100040E94232F089509
:1022D0001F93182F89E396E0612F0E94232F80918E
:1022E00000048127809300041F9108951F93192FE4
:1022F0000E946811812F0E9468111F910895DF923A
:10230000EF92FF920F931F93D82E7B01109200043F
:1023100009E316E0C80165EB0E94232FC80162E6BD
:102320000E94232F8D2D0E946811C7010E947611F3
:102330001F910F91FF90EF90DF900895E82FF0E04C
:10234000E456FC4FE185E03158F4F894F0E0EE0FEC
:10235000FF1FE95DFC4F0190F081E02D78940DC0E6
:10236000E03129F0E13129F0E0E0F2E006C082E15D
:1023700001C083E10E94702BFC01CF0108958EE023
:1023800060E00E94A12A8FE061E00E94A12A80E122
:1023900061E00E94A12A82E060E00E94A12A84E01C
:1023A00061E00E94A12A0895CF93DF93EC0100978A
:1023B00041F186E061E00E940D2B9E0140E050E07B
:1023C00068E478EE81E090E00E940B30C901DA0108
:1023D0008F3F9105A105B10531F028F08FEF90E016
:1023E000A0E0B0E008C00097A105B10521F481E0AC
:1023F00090E0A0E0B0E08093B3008091B0008061F5
:1024000007C086E060E00E940D2B8091B0008F7EB7
:102410008093B000DF91CF910895A0E2B0E0E3E1B6
:10242000F2E10C942E308CE00E94B40A882389F5E6
:1024300089E396E063E171E00E946B2D439A299A4B
:1024400080E00E949F0B0E947E0C4398299821C037
:1024500089E396E00E94EA2E482F8091C1048823E8
:1024600021F0842F0E948F0D14C080912C05E82F3D
:10247000F0E031969F012F713070319780912B05DC
:1024800090E02817390729F0EE5FFA4F4083209338
:102490002C0589E396E00E94B02E892BC9F6809125
:1024A0009A03843009F08EC00E941C2A6093B00405
:1024B0007093B1048093B2049093B30461157105D5
:1024C0008105910561F481E090E0A0E0B0E08093A7
:1024D000B0049093B104A093B204B093B30480917C
:1024E000BC049091BD0481609093BD048093BC04B2
:1024F00083E080939A038FE70E94900A09EF14E02B
:102500000E94A40AF80181938F01F5E002301F07B1
:10251000B9F74091E4048091F904282F30E0842F2A
:1025200090E08227932786FF40C080E448274093AD
:10253000E404C90188739070C89709F510E014C0CD
:102540001F5F8091F803E12FF0E084FF06C0E750A1
:10255000FB4F80810E94A10C07C0E750FB4F89E32D
:1025600096E060810E94232F212F30E08091F904B2
:1025700090E0877090708217930714F716C02F733E
:102580003070232B91F48091FA048093B4048091ED
:10259000FB048093B6048091FC048093B70480917F
:1025A000FF048093BE041092BF0480912D058130FA
:1025B00019F482E080932D0580912D05833011F46C
:1025C00010922D050E941C2A5B016C018091B804B9
:1025D0009091B904A091BA04B091BB040097A105F1
:1025E000B105C9F086017501E81AF90A0A0B1B0B3F
:1025F000D801C701885B9B40A040B04060F00E94BA
:10260000DB0A8093B5041092B8041092B9041092BA
:10261000BA041092BB0480ED93E00E94F50820916B
:10262000AC043091AD044091AE045091AF048601EA
:102630007501E21AF30A040B150BE616F7060807F4
:10264000190708F429C1A092AC04B092AD04C0925D
:10265000AE04D092AF04A8958091C0048830A0F059
:102660008091A1039091A203A091A303B091A40330
:10267000FCE1B695A79597958795FA95D1F70097C0
:10268000A105B10509F0A9C18091C0048F5F8093B5
:10269000C004E090B004F090B1040091B204109135
:1026A000B304E114F1040105110511F180ED93E08B
:1026B0000E94F508AE18BF08C00AD10A6A157B054A
:1026C0008C059D0588F48091A10384FD04C080EDF4
:1026D00097E00E94D4111092B0041092B1041092AD
:1026E000B2041092B30404C080E090E00E94D411C0
:1026F0009091E404907C9093E40400912C05109157
:102700002B050117B1F180912D05823091F590587C
:102710009093E40480ED93E00E94EB08893010F080
:1027200048E002C0482F415030E013C03F5FA32F64
:10273000B0E0812F90E0FC01EE5FFA4F2081FD01B7
:10274000EC51FB4F2083AE5DBA4F2C930196182FAE
:102750001F71341710F4101749F710932B05832FAE
:10276000895C9091E404892B8093E40430932205E2
:102770001AC020912D052430D1F490912205E3E276
:10278000F5E0A5EEB4E0292F30E02E0F3F1F02C088
:1027900081918D93E217F307D9F7995C8091E40456
:1027A000982B9093E40483E080932D0538C08091AA
:1027B000A704823061F491609093E404439A299ACB
:1027C00005EA13E07E010894E11CF11C11C090930E
:1027D000E40443982998222319F481E080932D057D
:1027E00080912D05833061F784E080932D05E8CF3B
:1027F000F80181918F010E949E11F70181939193BD
:102800007F01F3E0053B1F0799F78091F80387707C
:10281000BE016F5F7F4F45EE54E00E947C0985B199
:10282000846285B92091A5042223A1F09091DD0353
:10283000992381F08091A6048F5F8093A604815034
:10284000821729F41092A604892F815001C0892F84
:102850000E949A0B8091A4040E94C50A80ED93E027
:102860000E94EB08682F84EE94E00E948B0FE091A9
:10287000A404EF5FE093A404E83131F0F0E0E0530A
:10288000FC4F8785882341F41092A40405C0439A25
:10289000299A89E08093C0048091F803887171F1CE
:1028A00080919A03823051F58091BC049091BD04CF
:1028B000880F991F9093BD048093BC0483E080939C
:1028C0009A030E947E0C0E941C2A6093B8047093A5
:1028D000B9048093BA049093BB0461157105810516
:1028E000910561F481E090E0A0E0B0E08093B8044D
:1028F0009093B904A093BA04B093BB048091F803F9
:1029000084FF1EC08091BC049091BD048E7F0E9404
:102910003E0A182F8091B4046091BE040E94790D84
:10292000082F8091B504612F0E94790D282F809186
:10293000B6046091B704402F00919B030E940A11D6
:1029400085B18B7D85B98091A7048130D1F081302C
:1029500020F0823009F047C034C087E00E94402B4D
:10296000892B09F040C081E08093A7040E940E2AC1
:102970006093A8047093A9048093AA049093AB0475
:1029800032C087E00E94402B892B21F50E940E2A3D
:102990002091A8043091A9044091AA045091AB045D
:1029A000621B730B840B950B695E734080409040F3
:1029B000D0F082E08093A70480ED97E00E94D411CC
:1029C00012C087E00E94402B892B69F080E090E0E4
:1029D0000E94D4111092A70406C08091C0048830D0
:1029E00009F057CF54CFA096EAE00C944A3086E025
:1029F00061E00E94A12A86E060E00E940D2B82E047
:102A00008093B00085E08093B10083E061E00E9494
:102A1000A12A83E060E00E940D2B08951F93182FD8
:102A20000E941C2A60939F047093A0048093A104C9
:102A30009093A20410938D04112329F440E855E2E9
:102A400060E070E004C040E051EE60E070E089E3D7
:102A500096E00E94292E1F910895ACE1B0E0E3E3D7
:102A6000F5E10C942E300E941C2A7B018C0181E040
:102A70000E949F0B84E7A82E6E010894C11CD11CF4
:102A8000B3E0BB2EA982C60161E00E94C70FB092DD
:102A90009A030E947E0C6AEF70E080E090E00E9452
:102AA000422A80919A03833009F07DC089E396E041
:102AB0000E94B02E892B09F076C00E941C2A6E1944
:102AC0007F09800B910B6058734C894C914008F042
:102AD0006AC0D8CF8FE70E94900A0E94A40A84356A
:102AE00009F05CC089830E94A40A182F00E01093AB
:102AF0002404009323040E94A40A080F111D1093BC
:102B00002404009323040E94A40A809322040E94B8
:102B1000A40A80932104813108F040C0FF2407C03B
:102B20000E94A40A0F5F1B4FF8018083F3940F2DBE
:102B300010E08091210490E0880F991F0817190771
:102B400078F380E78983CE01019661E00E94C70F88
:102B500083E080939A030E947E0C62E370E080E041
:102B600090E00E94422A80919A038330A9F08FE777
:102B70000E94900A0E94A40A803581F4898305EBA3
:102B800013E00E94A40AF80181938F01F3E0003D55
:102B90001F07B9F781E003C082E001C083E06C96B3
:102BA000EAE00C944A3080919A03833009F092CF86
:102BB000F3CF83E00E94B40A8093F90384E00E947B
:102BC000B40A8093FA0387E061E00E94BA0A6AE0DF
:102BD00070E080E090E00E94422A0E947E0C00009B
:102BE00008950F931F93082F19C0439A299A64E6FA
:102BF00070E080E090E00E94422A4398299864E6C1
:102C000070E080E090E00E94422A1F5F101768F396
:102C10006CE271E080E090E00E94422A10E0F6CF82
:102C2000482F392F25E00DC0F999FECF1FBA842F08
:102C3000932F92BD81BD60BD0FB6F894FA9AF99AB0
:102C40000FBE215059F0F999FECF842F932F92BDDA
:102C500081BDF89A80B5681739F7089582E00E941F
:102C6000F1150895A0E0B0E0E8E3F6E10C94273018
:102C7000482E562EEE24FF2488249924C0E0D0E06C
:102C8000CC24DD2476E4372E04C055245394CC2480
:102C9000DD24442069F480919B03839DE00111248D
:102CA0006CE9E62E63E0F62E59E1852E912C1DC0CD
:102CB00021E0421671F480919B03839DE001112471
:102CC0006B9640EDE42E43E0F42E39E2832E912CF6
:102CD0000CC032E0431649F42BE9E22E23E0F22E39
:102CE00091E0892E912CC8E1D1E03E016C0C7D1C55
:102CF0001092360510923505E3011BC0552059F49A
:102D0000F999FECFD2BDC1BDF89A80B5F701E00FA9
:102D1000F11F808307C0F701E00FF11FCE01608132
:102D20000E9410160E0D1F1DF80180810E943008B0
:102D300021969E012619022F10E008151905F0F2C0
:102D4000CE015520D9F4F999FECFD2BDC1BDF89A74
:102D500020B5F999FECF2196D2BDC1BD2197F89A31
:102D600080B590E0B22EAA248A299B2920913505AE
:102D7000309136052817390759F487CF219660918D
:102D800036050E941016CE01609135050E9410167E
:102D900080E291E0C80ED91E91EEC91692E0D906E4
:102DA00008F477CF852DCDB7DEB7E1E10C94433041
:102DB00080E061E00E94321681E061E00E943216FC
:102DC000089582E061E00E943216089582E060E09A
:102DD0000E94321680919B03843020F010929B0356
:102DE0000E94E11608951F93182F0E94E616809105
:102DF0009B03811731F0143020F410939B030E9441
:102E0000E1161F91089510928B0485E6E6E2F4E046
:102E1000DF011D928A95E9F708951F93182F8F37C8
:102E200011F08830E1F5E0918B04EE2309F455C0F0
:102E3000E150E0938B04F0E0EA5DFB4F108289E300
:102E400096E06DE00E94232F10E00AC0E12FF0E031
:102E5000EA5DFB4F89E396E060810E94232F1F5FAC
:102E600080918B04181790F389E396E060E20E944A
:102E7000232F89E396E06DE00E94232F10E00AC023
:102E8000E12FF0E0EA5DFB4F89E396E060810E946C
:102E9000232F1F5F80918B04181790F31CC08B3178
:102EA00019F40E9403171FC08D30E9F08A30D9F061
:102EB00080918B04843688F489E396E0612F0E9428
:102EC000232F80918B04E82FF0E0EA5DFB4F108305
:102ED0008F5F80938B0480E007C089E396E067E012
:102EE0000E94D72BF8CF81E01F9108951F93CF93B5
:102EF000DF93CFEDD3E010E03BC089E396E062E2E0
:102F000071E00E94682D89E396E0612F4AE050E06D
:102F10000E94E52C89E396E06FE271E00E94682D43
:102F2000699170E080E090E02091DE0330E040E0C5
:102F300050E00E94B72F20E137E240E050E00E94CD
:102F4000B72FDC01CB014091D5035091D60360919E
:102F5000D7037091D803480F591F6A1F7B1F89E35D
:102F600096E02AE030E00E94AC2C1F5F183119F087
:102F70008881882311F6DF91CF911F910895EF92F8
:102F8000FF920F931F93882339F489E396E061E75A
:102F90007AE00E94F52B3BC090E00E94B20824E644
:102FA00030E040E050E00E94E92F122F032FF42E72
:102FB000E52E622F732F842F952F2AE030E040E01A
:102FC00050E00E94E92F89E396E0BA01A9012AE0C6
:102FD00030E00E949D2C89E396E06EE20E94D72BA0
:102FE000612F702F8F2D9E2D2AE030E040E050E0C1
:102FF0000E94E92FAB01BC0189E396E02AE030E0B2
:103000000E949D2C89E396E063E70E94092C1F91A2
:103010000F91FF90EF900895FF920F931F93CF931E
:10302000DF9389E396E067E67AE00E94B62B809111
:10303000B503813041F489E396E06EE47AE00E94C2
:10304000F52BFF246DC0823029F489E396E067E315
:103050007AE0F5CF843029F489E396E063E27AE000
:10306000EECF853071F789E396E068E17AE0E7CF4B
:10307000CF2DD0E0C930D1051CF06F2D685C02C0A7
:103080006F2D6F5C89E396E00E94D72B89E396E071
:1030900060E17AE00E94B62BBE016F5F7F4F89E34B
:1030A00096E04AE050E00E94412D89E396E065E019
:1030B0007AE00E94B62B8E010B541C4FD80111965A
:1030C000EC91E032F8F489E396E068EF79E00E9451
:1030D000B62BF8018181803130F089E396E063E31B
:1030E00071E00E94682DCB54DC4F698170E06F70F5
:1030F00070706F5F7F4F89E396E04AE050E00E9476
:10310000542D0DC0F0E0EF70F070EE0FFF1FE75B85
:10311000FC4F6081718189E396E00E946B2DF394EE
:1031200080912204F81608F4A3CF89E396E06DEDB0
:1031300079E00E94B62B8091CD030E94BF1789E3EE
:1031400096E062EC79E00E94B62B8091CE030E945B
:10315000BF1789E396E067EA79E00E94B62B809179
:10316000CF030E94BF1789E396E06CE879E00E94E4
:10317000B62B4091C5035091C6036091C70370916F
:10318000C803411551056105710539F189E396E0E0
:103190002AE030E00E94AC2C89E396E069E579E012
:1031A0000E94B62B8091C9030E94E508AB01BC01C7
:1031B00089E396E02AE030E00E94AC2C89E396E0B7
:1031C00065E379E00E94B62B89E396E06091CA033B
:1031D0004AE050E00E94F72C06C089E396E06CE2DA
:1031E00079E00E94F52B89E396E06FE079E00E9498
:1031F000B62B6091CB037091CC0389E396E04AE053
:1032000050E00E94D12C89E396E062EF78E00E94C2
:10321000B62B6091C403603450F470E06F5F7F4F51
:1032200089E396E04AE050E00E94542D06C089E30D
:1032300096E069EE78E00E94F52B89E396E06CEC6D
:1032400078E00E94B62B8091C30380FD03C065E344
:1032500071E002C069E371E089E396E00E946B2DA2
:1032600089E396E06FEA78E00E94B62B8091C30371
:1032700082700E94830D89E396E060E978E00E9405
:10328000B62B8091C30384700E94830D89E396E07E
:1032900061E778E00E94B62B8091C30388700E949A
:1032A000830DCDB7DEB7E5E00C944F301F93CF937D
:1032B000DF9389E396E06BEB7BE00E94B62B4091B5
:1032C000D5035091D6036091D7037091D80389E359
:1032D00096E02AE030E00E94AC2C89E396E065EAB3
:1032E0007BE00E94B62B4091D9035091DA036091A4
:1032F000DB037091DC0389E396E020E130E00E947B
:10330000AC2C89E396E06FE87BE00E94B62B89E362
:1033100096E06091DD034AE050E00E94F72C89E3DB
:1033200096E069E77BE00E94B62B89E396E0609126
:10333000DE034AE050E00E94F72C89E396E063E662
:103340007BE00E94B62BCFEDD3E010E012C011233A
:1033500031F089E396E06DE371E00E94682D89E326
:1033600096E069914AE050E00E94E52C1F5F183119
:1033700019F08881882359F789E396E00E94DF2BB2
:1033800089E396E06DE47BE00E94B62B89E396E04A
:103390006091F7034AE050E00E94F72C89E396E041
:1033A00068E37BE00E94B62BE091F803F0E0E77061
:1033B000F070EE0FFF1FE759FC4F6081718189E3C8
:1033C00096E00E946B2D89E396E063E27BE00E9429
:1033D000B62B8091F80390E0887190708830910549
:1033E00089F0893091051CF4892B39F01BC080319C
:1033F000910569F04897B1F40FC089E396E06AE15E
:103400007BE00EC089E396E06EE07BE009C089E3D3
:1034100096E068E07BE004C089E396E06EEF7AE036
:103420000E94F52B89E396E06AEE7AE00E94B62BC3
:103430004091D1035091D2036091D3037091D40392
:1034400089E396E02AE030E00E94AC2C89E396E024
:1034500061ED7AE00E94B62B8091A10380710E94F9
:10346000830D89E396E068EB7AE00E94B62B8091A9
:10347000A10380740E94830D89E396E06FE97AE0EE
:103480000E94B62B8091A10380720E94830D89E374
:1034900096E062E87AE00E94B62B80ED93E00E940D
:1034A000F508AB01BC0189E396E02AE030E00E9418
:1034B0009D2C89E396E06DE77AE00E94B62B80EDC3
:1034C00093E00E94F5089B01AC0160E472E48FE098
:1034D00090E00E94E92F89E396E0BA01A9012AE071
:1034E00030E00E949D2C89E396E06AE77AE00E9432
:1034F000F52BDF91CF911F910895EF92FF920F93DB
:103500001F937C0109E316E0C8016F2D70E04AE0CB
:1035100050E00E94C02CC8016EE20E94D72BB70178
:1035200084E0769567958A95E1F76F707070C801B1
:103530004AE050E00E94C02CC8016EE20E94D72BE6
:103540008FE0E822FF24C801B7014AE050E00E9462
:10355000C02C1F910F91FF90EF9008950F931F9330
:10356000CF93DF93209125042F3FA9F589E396E0BF
:1035700061EF75E00E94B62B83E793E00E947D1A0D
:1035800089E396E060ED75E00E94B62B80912304FC
:10359000909124040E947D1A89E396E06DE975E01C
:1035A0000E94F52B89E396E06AE775E00E94F52B0F
:1035B00089E396E062E675E00E94F52B89E396E0E8
:1035C0006DE375E00E94F52B89E396E00E94DF2B06
:1035D0000E940C1869C012160CF066C0332727FD34
:1035E00030958091220490E0821793070CF45CC020
:1035F00089E396E068E275E00E94B62B60912504AD
:10360000772767FD709589E396E04AE050E00E94D5
:10361000542D89E396E06DEF74E00E94B62B08E22A
:1036200010E03AC0C12FD0E0CC0FDD1FCF5FDB4FE1
:10363000288130E080912504992787FD9095019796
:103640002817390741F589E396E06FE371E00E949E
:10365000682D89E396E0602F4AE050E00E94E52C57
:1036600089E396E063E471E00E94682DE981F0E06F
:10367000EF70F070EE0FFF1FE75BFC4F6081718110
:1036800089E396E00E94682D89E396E067E471E0A3
:103690000E94682D0F5F1F5F80912104181710F2A0
:1036A00089E396E00E94DF2BDF91CF911F910F916C
:1036B0000895ACE1B0E0EFE5FBE10C943030282F49
:1036C000809125048F3F09F03BC1822F90E0FC01DF
:1036D0003A97EF36F10508F02CC1EC5CFF4F0C94E3
:1036E0005D3089E396E069E471E0A7C089E396E084
:1036F00065E571E00E946B2D85E78983DE011296F6
:10370000E5EBF3E08BE101900D928150E1F7CE0102
:1037100001966CE10E94C70F0E947E0C83E08093AB
:103720009A0368EC70E080E090E00E94422A809169
:103730009A03843009F0FDC08FE70E94900A0E942E
:10374000A40A8983853509F0F4C089E396E06FED1A
:1037500074E00E94F52B89E396E061EC74E00E942E
:10376000F52B89E396E063EA74E0ACC089E396E068
:103770006DE671E00E946B2D89E68983CE0101968A
:1037800061E00E94C70F0E947E0C83E080939A0341
:1037900068EC70E080E090E00E94422A80919A03F9
:1037A000843009F0C6C08FE70E94900A0E94A40AE4
:1037B00089838E010E5F1F4FBDE1EB2EF12CEC0EC5
:1037C000FD1E0E94A40AD8018D938D01AE15BF0580
:1037D000C1F7A5EBB3E0FE0132968BE101900D92AB
:1037E0008150E1F78981893409F0A3C089E396E02B
:1037F00065E874E00E94F52B89E396E067E674E0E3
:103800000E94F52B89E396E069E474E05BC089E3EC
:1038100096E067E871E00E946B2D8EEF809325049F
:1038200088C020522750922F9053809122048917EC
:1038300038F489E396E066E971E00E946B2D79C067
:10384000909325046FC084E18093250489E396E07A
:1038500062E174E037C085E18093250489E396E056
:103860006BED73E02FC086E18093250489E396E039
:1038700064EA73E027C087E18093250489E396E03A
:103880006AE573E01FC088E18093250489E396E030
:1038900069E473E017C089E18093250489E396E029
:1038A00065E373E00FC08AE18093250489E396E025
:1038B00060E273E007C08BE18093250489E396E022
:1038C00068EF72E00E94F52B34C089E396E06EED5C
:1038D00072E00E94F52B8091C30391E01DC089E343
:1038E00096E068EC72E00E94F52B8091C30392E0B1
:1038F00013C089E396E063EB72E00E94F52B8091A0
:10390000C30394E009C089E396E068E972E00E948D
:10391000F52B8091C30398E089278093C3038FEF31
:10392000809325040E94AE1A04C089E396E00E94A9
:10393000EA2E89E396E00E94B02E892BB1F762C18E
:10394000822F0E940D17882309F45CC180918B049B
:10395000882321F48FEF809325044CC186E294E004
:1039600060E070E040E050E00E94A2069B01AC01E4
:1039700060912504862F992787FD9095A92FB92F4F
:10398000FC013197EB31F10508F024C1ED55FF4FF3
:103990000C945D30E62FFF27E7FDF095809122041F
:1039A00090E08E179F070CF415C1DA01C901019749
:1039B000A109B1098097A105B10548F0A8E2FA2E46
:1039C00000E010E06F010894C108D10825C0EB5455
:1039D000FC4F822F81508083E5C0612F70E0660F1D
:1039E000771F6F5F7B4FFB01808190E08C159D05F9
:1039F00091F48F2D90E0A0E0B0E082179307A40728
:103A0000B50741F4F601EB54FC4FDB0111968C91A4
:103A1000818301E0F3941F5F809121041817E8F27D
:103A2000BFC02F3F31054105510511F008F0D2C04C
:103A30002093CD03B7C02F3F31054105510511F04B
:103A400008F0C8C02093CE03ADC02F3F310541051B
:103A5000510511F008F0BEC02093CF03A3C08091A0
:103A600026048062803719F587E294E060E070E018
:103A700040E050E00E94A2069B01AC01DC01CB01BA
:103A80000197A109B1090897A105B10508F0B5C0D2
:103A9000CA01B90124ED30E340E050E00E94B72FA5
:103AA0009B01AC012A5E3C4A4A46554E24C08636EC
:103AB00011F587E294E060E070E040E050E00E94A1
:103AC000A2069B01AC01DC01CB010197A109B10960
:103AD0000797A105B10508F090C0CA01B90128EA0D
:103AE00031E640E050E00E94B72F9B01AC01245E1C
:103AF0003C434E46544E211531054105510561F0B8
:103B0000DA01C90180509447AB48B24381509A45CD
:103B1000A246B24008F05EC02093C5033093C603AE
:103B20004093C7035093C8033DC02F3F3105410563
:103B3000510511F008F04EC02093C90333C0DA01DB
:103B4000C9010197A109B1098F3F9105A105B105EF
:103B500008F040C02093CA0325C0DA01C901845C83
:103B60009940A040B0408D549D41A040B04030F4F9
:103B70003093CC032093CB0301E001C000E021157A
:103B800031054105510511F48FEF07C0213431058E
:103B90004105510528F4822F81508093C40302C04F
:103BA0000023C1F080918C048823D1F48091D90343
:103BB0009091DA03A091DB03B091DC030196A11D83
:103BC000B11D8093D9039093DA03A093DB03B093E4
:103BD000DC0306C089E396E068EA71E00E946B2D81
:103BE0000E9403178FEF8093250489E396E06AE033
:103BF0000E94092C0E94AE1A05C021E030E040E08E
:103C000050E07ECF6C96E8E00C944C3089E396E06F
:103C10006CE472E00E94F52B89E396E064E372E0C5
:103C20000E94F52B89E396E00E94B02E892B31F09B
:103C300089E396E00E94EA2E0E94591B0E942D15EE
:103C4000823019F0833069F405C089E396E066E1BB
:103C500072E004C089E396E06FEF71E00E94F52BFB
:103C600008958FEF8093250410928C040E94AE1A61
:103C70000CC089E396E00E94B02E892B31F089E3D5
:103C800096E00E94EA2E0E94591B809125048E3FE7
:103C900081F7089580912504992787FD9095A92F94
:103CA000B92FFC013196EB30F10508F074C0E254F5
:103CB000FF4F0C945D3089E396E064E678E00E9463
:103CC000F52B83E793E00E947D1A89E396E06CE48C
:103CD00078E00E94F52B89E396E067E278E00E94A5
:103CE000F52B89E396E06DEF77E00E94F52B89E3F1
:103CF00096E06CED77E00E94F52B89E396E06FEAA1
:103D000077E00E94F52B89E396E069E877E00E946E
:103D1000F52B89E396E065E677E00E94F52B89E3D1
:103D200096E06EE377E00E94F52B89E396E00E942F
:103D3000DF2B0E9456192FC089E396E061E277E0FD
:103D400028C089E396E06CEF76E023C089E396E033
:103D500067EE76E01EC089E396E068EC76E019C075
:103D600089E396E064E876E014C089E396E06FE6C4
:103D700076E00FC089E396E06AE576E00E94F52BD5
:103D800089E396E064E176E004C089E396E06EEFB3
:103D900075E00E94F52B6AE070E080E090E00E9400
:103DA000422A04C089E396E00E94EA2E89E396E065
:103DB0000E94B02E892BB1F70895A2E2B0E0E3EEA5
:103DC000FEE10C9426308E010F5F1F4F80E1D80179
:103DD0001D928A95E9F789E396E066EC71E00E940E
:103DE0006B2D0E94D91520E034E74BE852E32F8F6A
:103DF00038A349A35AA380E09EECADEEB4E38B8FC9
:103E00009C8FAD8FBE8F24EF31E040E050E02F8BD0
:103E1000388F498F5A8F30E5C32E33ECD32EE12CE7
:103E2000F12C412C24E7522E2BE8622E22E3722E35
:103E300088249924540133241E8A1D8A198A1A8AD7
:103E40001B8A1C8AFFC089E396E00E94EA2E843414
:103E5000B9F0853430F48332B9F18C3209F0CCC03A
:103E600044C0833509F0C8C02F8D38A149A15AA19B
:103E7000C901DA012C013D01882499245401E2C0D2
:103E800089E396E064E40E94D72B89E396E040E062
:103E900054E76BE872E32AE030E00E940B2D89E3DF
:103EA00096E06CE20E94D72B89E396E040E05EEC5E
:103EB0006DEE74E32AE030E00E940B2D89E396E07A
:103EC0006CE20E94092CBEC019821A821B821C82DD
:103ED0001D821E821F82188619861A861B861C86E2
:103EE0001D861E861F86188A3AC0339434E0331626
:103EF00009F0A8C069817A818B819C8128EE33E02A
:103F000040E050E00E94B72F6F8F78A389A39AA357
:103F10006D817E818F8198850E94B72F6B8F7C8FFA
:103F20008D8F9E8F89859A85AB85BC858F8B988F69
:103F3000A98FBA8F6D857E858F8598890E94B72F4E
:103F40006B017C0190E2C9169EE4D90690E0E90677
:103F500090E0F90630F48CE162E30E94BA0A33245F
:103F600071C0A0E3CA16A5E7DA06A0E0EA06A0E061
:103F7000FA0618F48CE162E2F0CFB0E4CB16BCE9AB
:103F8000DB06B0E0EB06B0E0FB0618F48CE166E27D
:103F9000E4CFE0E5CE16E3ECDE06E0E0EE06E0E09E
:103FA000FE0618F48CE162E1D8CFF0E6CF16FAEE07
:103FB000DF06F0E0EF06F0E0FF0618F48CE165E1C3
:103FC000CCCF20E7C21621E1D20621E0E20620E0B4
:103FD000F20618F48CE161E0C0CF30EAC31636E88F
:103FE000D30631E0E30630E0F30618F48CE163E039
:103FF000B4CF8CE165E0B1CF90ED292E280E49E0D9
:10400000421500F1032D10E0000F111F000F111FCA
:1040100081E090E08C0F9D1F080F191FD8016D9152
:104020007D918D919C912AE030E040E050E00E942B
:10403000B72F620D711D811D911DF8016083718381
:104040008283938389E396E00E94B02E892B09F046
:10405000FACE81149104A104B10489F4C301B20120
:104060000E94300B61E070E080E090E00E94422A04
:10407000FFEFFE8B1D8A198A1A8A1B8A1C8A2F89D8
:10408000388D498D5A8D82169306A406B506E0F444
:104090000E94DB0A29893A894B895C89280F311DE6
:1040A000411D511D298B3A8B4B8B5C8B3D893817F9
:1040B00008F48D8B4E89841708F48E8B0894811C2C
:1040C000911CA11CB11C56C0C301B20128EE33E003
:1040D00040E050E00E94E92F89E396E0BA01A9018F
:1040E0002AE030E00E949D2C89E396E06CE20E9479
:1040F000D72B89E396E06D894AE050E00E94E52CD9
:1041000089E396E06CE20E94D72B69897A898B89D2
:104110009C89A50194010E94E92F89E396E0BA01E8
:10412000A9012AE030E00E949D2C89E396E06CE230
:104130000E94D72B89E396E06E894AE050E00E9406
:10414000E52C89E396E06CE20E94092C4C0C5D1C86
:104150006E1C7F1C8B8D9C8DAD8DBE8D8415950541
:10416000A605B70520F44F8C58A069A07AA0882432
:10417000992454012F8D38A149A15AA1285E3340BA
:104180004040504009F05ECFA296E2E10C944230EC
:10419000A0E0B0E0EEECF0E20C9431300E941C2A7A
:1041A0006115710581059105C9F30E949906109268
:1041B000D9031092DA031092DB031092DC03DD24A2
:1041C000E090D903F090DA030091DB031091DC0357
:1041D000102F0F2DFE2CEE240E9494062FEF30E0BE
:1041E00040E050E00E940B30E60EF71E081F191F3A
:1041F000E092D903F092DA030093DB031093DC031F
:10420000D39444E0D416E1F6CFEDD3E000E010E023
:1042100040E1E42E47E2F42E4EC00F5F19F40E94F5
:104220004D084DC00E94940622E330E040E050E08B
:104230000E940B306F5FEFEDF3E090E004C08191DE
:10424000861759F39F5F9117D0F38091DE0390E0BA
:104250008E9D90018F9D300D9E9D300D1124862FD7
:1042600090E0AC01249FC001259F900D349F900DDC
:104270001124AA2797FDA095BA2F2091D50330913C
:10428000D6034091D7035091D803820F931FA41FE8
:10429000B51F20919D0330919E0340919F03509143
:1042A000A003281739074A075B0708F4B6CF6993BC
:1042B0001F5F183121F08881882309F0AECFCDB778
:1042C000DEB7E7E00C944D3080E060E00E943216EB
:1042D000882331F081E060E00E943216882341F4A7
:1042E0000E9492080E944D080E94C8200E94D81681
:1042F0000895AAE5B0E0EFE7F1E20C9432308B01CB
:104300007A018B3009F426C18C3040F5853009F4F0
:1043100084C0863080F4823009F459C0833020F4A0
:10432000813009F050C242C0833009F461C084304A
:1043300009F049C265C0883009F49DC0893038F45D
:10434000863009F486C0873009F03DC28CC08930C0
:1043500009F499C08A3009F036C2C9C0893609F417
:1043600082C18A3680F4863609F42DC1873620F45E
:10437000853609F028C20EC1873609F43DC188365A
:1043800009F021C241C18C3609F4C4C18D3638F41C
:104390008A3609F473C18B3609F015C2AFC18D3668
:1043A00009F4ECC1873C09F00EC200C281E069E269
:1043B00070E00E947F1100ED13E0F80181918F0100
:1043C0000E946811F3E0093F1F07B9F704C282E0B9
:1043D0006BE170E00E947F1105EB13E0F801819121
:1043E0008F010E946811F3E0003D1F07B9F7F3C188
:1043F00083E061E070E00E947F110E942D15E9C109
:1044000084E061E070E00E947F1181E00E94681109
:104410000E9461110E94DD1EE0C16091210470E0E4
:10442000660F771F85E00E947F1100E010E008C052
:10443000F801EF5FFB4F80810E9468110F5F1F4FF3
:104440008091210490E0880F991F0817190780F3C5
:10445000C2C186E062E070E00E947F1183E793E0D2
:104460000E947611B8C187E061E070E00E947F1180
:1044700080912204AEC188E061E070E00E947F116B
:1044800080919B03A6C186E68983CE01019661E0F7
:104490000E94C70F0E947E0C83E080939A0368EC11
:1044A00070E080E090E00E94422A80919A0384307C
:1044B000E1F48FE70E94900A0E94A40A898386345F
:1044C00071F489E060E270E00E947F1110E00E94C8
:1044D000A40A0E9468111F5F1032C9F77CC189E0ED
:1044E00061E070E00E947F11C7C089E06DC18AE081
:1044F00069E170E00E947F1181E080939C038091CC
:10450000A305882351F08091A1039091A203A0916B
:10451000A303B091A403806809C08091A103909186
:10452000A203A091A303B091A4038F778093A1036A
:104530009093A203A093A303B093A4030CE913E008
:10454000F80181918F010E946811F3E0053B1F077C
:10455000B9F741C18BE061E270E00E947F11809168
:10456000C0048F3F39F08091C0048F5F8093C004F6
:10457000815002C08091C0040E94681110E0812F18
:104580000E949E110E94190A0E9476111F5F10312D
:10459000B1F721C185E661E070E00E947F11093228
:1045A000110509F015C120E030E0F901E053FC4F9E
:1045B000D701A20FB31F8C9180832F5F3F4F293209
:1045C000310599F759C086E661E070E00E947F11DD
:1045D0000B31110509F0FCC020E030E0F901EB548B
:1045E000FC4FD701A20FB31F8C9180832F5F3F4FE9
:1045F0002B31310599F740C087E661E070E00E94F9
:104600007F110E94D81638C088E661E070E00E94F1
:104610007F1185E78A83DE011396E5EBF3E08BE1FA
:1046200001900D928150E1F7CE0102966CE10E945B
:10463000C70F0E947E0C83E080939A0360E273E0D0
:1046400080E090E00E94422A80919A03843009F031
:10465000BFC08FE70E94900A0E94A40A8A83853512
:1046600009F0B6C009C089E661E070E00E947F11E0
:104670000E944D080E94920881E0ABC08AE661E08A
:1046800070E00E947F1189E68E8FCE014E9661E028
:104690000E94C70F0E947E0C83E080939A0360E221
:1046A00073E080E090E00E94422A80919A03843077
:1046B00009F08EC08FE70E94900A0E94A40A8E8F94
:1046C0008E01015E1F4F6AE3E62EF12CEC0EFD1EFB
:1046D0000E94A40AF80181938F01EE15FF05C1F72E
:1046E000A5EBB3E0FE017F968BE101900D92815026
:1046F000E1F78E8D893409F06BC0BECF8BE661E0A7
:1047000070E00E947F11F70180810E94F3160E94E1
:104710006421B2CF8CE661E070E00E947F1100322C
:10472000110571F487E68AAFDE01DB96F70180E2BE
:1047300001900D928150E1F7CE01CA9661E205C069
:1047400087E48AAFCE01CA9661E00E94C70F0E943B
:104750007E0C83E080939A036CE474E080E090E048
:104760000E94422A80919A03843091F58FE70E943B
:10477000900A0E94A40A873459F57ECF8DE661E045
:1047800070E00E947F110931110511F520E030E041
:10479000F901E456FC4FD701A20FB31F8C9180831F
:1047A0002F5F3F4F2931310599F766CF87EC61E0E4
:1047B00070E00E947F1181E00E9468110E946111E7
:1047C0001092FF030AC08AEC61E070E00E947F1142
:1047D00080E00E9468110E946111C65ADF4FE6E036
:1047E0000C944E30A0E0B0E0E8EFF3E20C942E30F1
:1047F00084E0A82E06E0B02E15E0C12E07E315E0F8
:10480000B4E6DB2EA2E0EA2EF3E0FF2EA1C089E39E
:1048100096E00E94EA2E982F8093A2058091A10530
:10482000833021F1843028F4813099F08230B8F45B
:1048300009C0853009F448C0853020F1863009F080
:1048400087C05FC0953B09F083C081E08093A105DC
:104850007FC0923609F07AC0E092A10579C09093AA
:10486000A00590939F05F092A10572C090939D05BD
:1048700010929E0580919F05892780939F05A092A5
:10488000A10566C0D92FC0E020919D0530919E05FD
:104890002C2B3D2B30939E0520939D0580919F05E9
:1048A000892780939F05C092A1052536310508F41C
:1048B0004FC08CEC61E070E00E947F1181E00E94AB
:1048C00068110E94611142C020919B0530919C05A6
:1048D000F901E95CFA4F908380919F0589278093C5
:1048E0009F052F5F3F4F30939C0520939B05809140
:1048F0009D0590919E052817390750F1B092A105AA
:1049000027C080919F05891759F460919B0570918C
:104910009C058091A00547E355E00E9479210DC0D8
:104920008BEC62E070E00E947F118091A0050E94F4
:104930006811809100040E946811F8018D2D119278
:104940008A95E9F710929C0510929B051092A1059B
:1049500089E396E00E94B02E892B09F058CFCDB79D
:10496000DEB7EAE00C944A3081E08093FF0308C090
:1049700089E396E00E94B02E892B11F00E94F22369
:104980008091FF038823A1F708951F9310912504B8
:104990001F3F09F0F1C0893409F467C08A3428F553
:1049A000883309F479C0893368F4803309F486C008
:1049B000813308F06FC08B3109F44DC0813209F0AA
:1049C000D5C03DC0813409F49AC0823438F48933AB
:1049D00009F472C0803409F0C9C031C0823409F4CE
:1049E000A1C0863409F0C2C052C0823609F49AC010
:1049F000833690F4883579F1893538F4823509F4B5
:104A00003FC0833509F0B2C01FC08A3509F4A9C080
:104A1000813609F0ABC073C0823791F1833730F42F
:104A20008636A9F1893609F0A1C01FC0883799F0F0
:104A30008A3709F496C0833709F098C005C089E326
:104A400096E069E471E019C00E94D81689E396E007
:104A500063ED71E006C00E94642189E396E06DEE8B
:104A600071E00E946B2D8EEF7FC00E944D080E9466
:104A7000920889E396E06CE072E00E946B2D76C0AC
:104A80000E94C82089E396E065E272E0F6CF0E94BA
:104A900076176CC0805368C089E396E06CEE71E0D5
:104AA0000E94F52B9091F803892F885F8871977E7B
:104AB000892B8093F80320C089E056C089E396E0F3
:104AC00069ED71E00E94F52B8091A1039091A20302
:104AD000A091A303B091A40320E130E040E050E0B6
:104AE00082279327A427B5278093A1039093A2033D
:104AF000A093A303B093A4031093250437C089E3C4
:104B000096E063EC71E00E94F52B8091A1039091F7
:104B1000A203A091A303B091A40320E430E040E0FD
:104B200050E012C089E396E062EB71E00E94F52B41
:104B30008091A1039091A203A091A303B091A4033B
:104B400020E230E040E050E082279327A427B527F9
:104B50008093A1039093A203A093A303B093A40313
:104B600002C00E94061E8FEF8093250480912504C9
:104B70008E3F09F4DDC0D4C00E940D17882309F4CC
:104B8000D7C080918B04882321F48FEF8093250474
:104B9000C7C086E294E060E070E040E050E00E9430
:104BA000A2069B01AC0180912504992787FD909571
:104BB000A92FB92FFC013197E930F10508F08CC01D
:104BC000E753FF4F0C945D30DA01C90181509447DF
:104BD000AB48B2438F5F9945A246B24008F07CC013
:104BE0002093D5033093D6034093D7035093D80333
:104BF0009AC02093D9033093DA034093DB03509398
:104C0000DC0381E080938C048EC02830310541059F
:104C1000510508F061C02093DD0385C0DA01C901A8
:104C20000197A109B1090A97A105B10508F054C07F
:104C30002093DE0378C086E294E06DE371E00E9489
:104C4000BE0710E00EC0183130F4E12FF0E0E05361
:104C5000FC4F87871F5F80E090E06DE371E00E946A
:104C6000BE07009759F00E94A007009761F706C0A1
:104C7000E12FF0E0E053FC4F17861F5F1831C0F3BF
:104C800052C0253031054105510530F52093F70319
:104C90004AC0DA01C9010197A109B1090697A10526
:104CA000B105D0F48091F803887F822B8093F803BC
:104CB0003AC0DA01C9010197A109B1098050924CAB
:104CC000A140B04048F42093D1033093D2034093E5
:104CD000D3035093D40327C089E396E068EA71E0D8
:104CE0000E946B2D13C08091D9039091DA03A0919B
:104CF000DB03B091DC030196A11DB11D8093D903A4
:104D00009093DA03A093DB03B093DC030E940317B4
:104D10008FEF8093250489E396E06AE00E94092CD6
:104D20000E944A1E05C080918C048823E1F2EECFD8
:104D30001F9108958FEF8093250410928C040E9498
:104D40004A1E0CC089E396E00E94B02E892B31F0F8
:104D500089E396E00E94EA2E0E94C52480912504F2
:104D60008E3F81F76AE070E080E090E00E94422A86
:104D700004C089E396E00E94EA2E89E396E00E944F
:104D8000B02E892BB1F70895AAE2B0E0EAECF6E282
:104D90000C942B300E940E2A7B018C0181E00E9432
:104DA0009F0B04C089E396E00E94EA2E89E396E017
:104DB0000E94B02E892BB1F743982998DD24D39413
:104DC00032E6732E22E0822E912C8C0E9D1E5E0107
:104DD0000894A11CB11C93E0C92E0E940E2A20E069
:104DE00030E06E197F09800B910B693C71058105DC
:104DF000910510F021E030E08D2D90E0282339233B
:104E0000232BB9F10E940E2A7B018C0185B18462AB
:104E100085B980ED97E00E94D4117982D401E0ED4C
:104E2000F3E089E201900D928150E1F7C5016AE259
:104E30000E94C70F85B18B7D85B980E090E00E940C
:104E4000D411C0929A030E947E0C62E370E080E06D
:104E500090E00E94422A80919A03843051F4C092DB
:104E60009A038FE70E94900A0E94A40A823409F4F0
:104E7000DD2487E00E94402B892B79F5DD24D39433
:104E80002CC0439A299A85B1846285B989E396E05A
:104E90000E94EA2E8D30910569F08E3091051CF448
:104EA0000A97B1F407C08332910569F08234910505
:104EB00079F40CC089E396E064EA71E00E94F52B76
:104EC0000E949A2605C00E94DD1E02C00E94B424E2
:104ED0004398299885B18B7D85B989E396E00E9436
:104EE000B02E892B09F479CFCCCF8F929F92AF92BD
:104EF000BF92CF92DF92EF92FF920F931F9387E0C2
:104F00000E94402B892B09F083C068EC70E080E0A0
:104F100090E00E94422A80E090E00E94D4110E941A
:104F20000E2A5B016C0140ECE42E42E1F42E012DCF
:104F3000112DE60EF71E081F191F06C087E00E94FC
:104F4000402B892B09F062C00E940E2A6E157F0546
:104F50008007910798F387E00E94402B892B09F086
:104F600055C080ED97E00E94D4110E940E2A7B016B
:104F70008C0199249394882488E496E2A0E0B0E020
:104F8000A80EB91ECA1EDB1E29C0AE14BF04C0067F
:104F9000D10638F480ED97E00E94D41188248394E0
:104FA0001DC00E940E2A6E197F09800B910B693C6F
:104FB00071058105910590F00E940E2A7B018C01FC
:104FC00080E0992009F481E0982E882319F480E08C
:104FD00090E002C080ED97E00E94D41187E00E942B
:104FE000402B892B91F280E090E00E94D411882020
:104FF00049F080919B038F5F83700E94F3160E949B
:10500000642106C00E94C8200E94D8160E94C426AF
:105010001F910F91FF90EF90DF90CF90BF90AF90D6
:105020009F908F90089580E06DEF77E042E050E030
:105030000E9449290895EF92FF920F931F9380E0F9
:105040000E9419080E94BF1181E161E00E94A12A1B
:105050008DE061E00E94A12A89E061E00E94A12A1E
:105060008AE061E00E94A12A87E060E00E94A12A14
:1050700088E060E00E94A12A88E061E00E940D2B98
:105080000E94F71489E396E040E052EC61E070E0A2
:105090000E94292E0E94E6160E9464210E945E0D45
:1050A0008FEF8093C0040E94132878940E940E2AE8
:1050B0007B018C018091C0048F3F09F0DFC00E940A
:1050C0000E2A6E197F09800B910B605D774080403E
:1050D000904008F0D3C0EECF89E396E00E94EA2E1C
:1050E00089E396E00E94B02E892BB1F789E396E020
:1050F00062E472E00E94682D83E793E00E947D1ACB
:1051000089E396E069E572E00E94682D89E396E004
:1051100063E070E04AE050E00E94542D62E370E0EA
:1051200080E090E00E94422A89E396E00E94B02E3F
:1051300004970CF189E396E00E94EA2E82349105EF
:10514000D1F489E396E00E94EA2E8E34910599F419
:1051500089E396E00E94EA2E8434910561F489E3A4
:1051600096E00E94EA2E819731F480E090E00E9460
:10517000D4110E94C4264091D1035091D203609172
:10518000D3037091D403DB01CA010197A109B109CE
:105190000497A105B10568F44093C104433029F098
:1051A00040E052EC61E070E004C040EA56E861E0A3
:1051B00070E089E396E00E94292E0E9475274398AB
:1051C000299880E090E00E94D4110E945E0D109218
:1051D000A5048091A10383FF11C08091E50388237A
:1051E00051F08091EC03882331F08091F303882300
:1051F00011F087E001C085E08093A50480E00E9463
:105200009F0B8091A4040E94C50A0E947E0C1092FC
:105210002B0510922C0510922D0510E015C062E3AD
:1052200070E080E090E00E94422A80ED97E00E94CA
:10523000D41162E370E080E090E00E94422A80E0B6
:1052400090E00E94D4111F5F80919B03811738F773
:105250008091F80390E084FF09C020E0887190708D
:10526000489709F421E0822F0E940E158FE00E94DA
:1052700019081F910F91FF90EF90089580ED97E02E
:105280000E94D41187E061E00E940D2B439A299A75
:1052900027CF823000F5E82FF0E0EE0FFF1FEC552E
:1052A000FA4F71836083882319F08130A1F408C01C
:1052B000809169008C7F842B80936900E89A08951F
:1052C00080916900440F551F440F551F837F842B25
:1052D00080936900E99A08951F920F920FB60F927A
:1052E00011242F933F934F935F936F937F938F93EB
:1052F0009F93AF93BF93EF93FF938091A4059091F9
:10530000A505892B29F0E091A405F091A505099543
:10531000FF91EF91BF91AF919F918F917F916F918D
:105320005F914F913F912F910F900FBE0F901F9063
:1053300018951F920F920FB60F9211242F933F933F
:105340004F935F936F937F938F939F93AF93BF938D
:10535000EF93FF938091A6059091A705892B29F0E3
:10536000E091A605F091A7050995FF91EF91BF91F6
:10537000AF919F918F917F916F915F914F913F91ED
:105380002F910F900FBE0F901F9018951F920F92A4
:105390000FB60F9211242F933F938F939F93AF9348
:1053A000BF938091AC059091AD05A091AE05B091F1
:1053B000AF053091B0050196A11DB11D232F2D5FC2
:1053C0002D3720F02D570196A11DB11D2093B0055A
:1053D0008093AC059093AD05A093AE05B093AF0557
:1053E0008091A8059091A905A091AA05B091AB055F
:1053F0000196A11DB11D8093A8059093A905A093C6
:10540000AA05B093AB05BF91AF919F918F913F914A
:105410002F910F900FBE0F901F9018958FB7F89493
:105420002091AC053091AD054091AE055091AF058E
:105430008FBFB901CA0108959FB7F8942091A805BC
:105440003091A9054091AA055091AB0586B5A89B5E
:1054500006C08F3F21F02F5F3F4F4F4F5F4F9FBFE1
:10546000542F432F322F2227280F311D411D511D4C
:1054700082E0220F331F441F551F8A95D1F7B901CF
:10548000CA010895EF92FF920F931F93CF93DF937A
:105490007B018C010E941C2AEB010EC00E941C2A79
:1054A0006C1B7D0B685E7340C8F30894E108F1083B
:1054B00001091109C851DC4FE114F104010511057E
:1054C00069F7CDB7DEB7E6E00C944E30789484B53A
:1054D000826084BD84B5816084BD85B5826085BDF0
:1054E00085B5816085BDEEE6F0E0808181608083D6
:1054F000E1E8F0E0108280818260808380818160B9
:105500008083E0E8F0E0808181608083E1EBF0E07F
:10551000808184608083E0EBF0E080818160808323
:10552000EAE7F0E08081846080838081826080830C
:105530008081816080838081806880831092C10037
:105540000895CF93DF93482F50E0CA018D5F934FAA
:10555000FC0134914151544FFA018491882369F13F
:1055600090E0880F991FFC01EF52F44FA591B49180
:10557000FC01E552F44FC591D491662351F42FB745
:10558000F8948C91932F909589238C93888189230B
:105590000BC0623061F42FB7F8948C91932F9095E3
:1055A00089238C938881832B88832FBF06C09FB764
:1055B000F8948C91832B8C939FBFDF91CF910895AA
:1055C000833071F0843028F48130A1F0823021F5ED
:1055D00014C08630B1F08730D1F08430E9F404C0D3
:1055E000809180008F7703C0809180008F7D8093B1
:1055F0008000089584B58F7702C084B58F7D84BD07
:1056000008958091B0008F778093B00008958091C5
:10561000B0008F7D8093B0000895FF920F931F9389
:10562000F62E482F50E0CA01895E934FFC01249169
:10563000CA018D5F934FFC0114914151544FFA01FF
:1056400004910023C9F0222319F0822F0E94E02A3E
:10565000E02FF0E0EE0FFF1FE552F44FA591B4915B
:105660009FB7F894FF2021F48C911095812302C0FC
:105670008C91812B8C939FBF1F910F91FF90089568
:105680000F931F93482F50E0CA01895E934FFC018E
:105690002491CA018D5F934FFC0104914151544FF5
:1056A000FA011491112319F420E030E015C02223EF
:1056B00019F0822F0E94E02A812F90E0880F991F15
:1056C0008B51944FFC01A591B4918C9120E030E076
:1056D000802311F021E030E0C9011F910F9108955E
:1056E000982F8E3008F09E509770809148038295D5
:1056F000880F880F807C892B80937C0080917A00B2
:10570000806480937A0080917A0086FDFCCF20919E
:10571000780040917900942F80E030E0282B392BDD
:10572000C9010895A0E0B0E0E8E9FBE20C94303054
:105730007C016B018A01C0E0D0E00FC0D6016D9101
:105740006D01D701ED91FC910190F081E02DC70131
:105750000995C80FD91F015010400115110571F7A7
:10576000CE01CDB7DEB7E8E00C944C30EF92FF925B
:105770000F931F93CF93DF937C018B01C0E0D0E0A8
:10578000F8010F5F1F4F6491662359F0D701ED9127
:10579000FC910190F081E02DC7010995C80FD91F38
:1057A000EFCFCE01CDB7DEB7E6E00C944E30DC0192
:1057B000ED91FC910190F081E02D09950895EF9213
:1057C000FF920F931F938C016DE00E94D72B7C01F9
:1057D000C8016AE00E94D72B9C012E0D3F1DC90114
:1057E0001F910F91FF90EF900895EF92FF920F930A
:1057F0001F937C010E94B62B8C01C7010E94DF2BF6
:105800009C01200F311FC9011F910F91FF90EF9054
:105810000895EF92FF920F931F937C010E94D72B64
:105820008C01C7010E94DF2B9C01200F311FC90191
:105830001F910F91FF90EF900895CF93DF93EC01AC
:105840006115710519F420E030E00FC0DB010D9007
:105850000020E9F71197A61BB70BE881F9810280B8
:10586000F381E02DAD0109959C01C901DF91CF9134
:1058700008954F925F927F928F929F92AF92BF92C4
:10588000CF92DF92EF92FF920F931F93DF93CF930C
:10589000CDB7DEB7A1970FB6F894DEBF0FBECDBF70
:1058A0002C01742ECB01223008F42AE019A231E237
:1058B000C32ED12CCC0EDD1E822E9924AA24BB240B
:1058C000672D752FA50194010E94E92F79018A01A6
:1058D000C801B701A50194010E94B72F472D461BAF
:1058E0000894C108D1084A3010F4405D01C0495CF9
:1058F000F6014083E114F1040105110521F07E2C2D
:105900005F2DC801DDCFC201B6010E941D2CA196FA
:105910000FB6F894DEBF0FBECDBFCF91DF911F91C0
:105920000F91FF90EF90DF90CF90BF90AF909F903E
:105930008F907F905F904F900895DC012115310585
:1059400041F4ED91FC910190F081E02D642F0995D7
:1059500008950E94392C0895EF92FF920F931F93A0
:105960007C010E949D2C8C01C7010E94DF2B9C01B1
:10597000200F311FC9011F910F91FF90EF900895E3
:10598000EF92FF920F931F939A017B0100E010E0CA
:10599000B801A7010E949D2C1F910F91FF90EF90DD
:1059A0000895EF92FF920F931F937C010E94C02CE9
:1059B0008C01C7010E94DF2B9C01200F311FC90100
:1059C0001F910F91FF90EF900895EF92FF920F9328
:1059D0001F939A01E62EFF2400E010E0B801A70112
:1059E0000E949D2C1F910F91FF90EF900895EF92D0
:1059F000FF920F931F937C010E94E52C8C01C7013D
:105A00000E94DF2B9C01200F311FC9011F910F91B4
:105A1000FF90EF900895A0E0B0E0E1E1FDE20C948A
:105A20003030EC016A017B012115310541F4E88138
:105A3000F9810190F081E02D642F09951BC02A3077
:105A40003105B1F477FF13C06DE20E94D72B8C01B2
:105A500044275527BA014C195D096E097F09CE010B
:105A60002AE00E94392C9C01200F311F04C02AE03B
:105A70000E94392C9C01C901CDB7DEB7E8E00C9437
:105A80004C30EF92FF920F931F937B019A010027F6
:105A9000F7FC0095102FB801A7010E940B2D1F9154
:105AA0000F91FF90EF900895EF92FF920F931F9345
:105AB0007C010E94412D8C01C7010E94DF2B9C01BB
:105AC000200F311FC9011F910F91FF90EF90089592
:105AD0000E941D2C0895EF92FF920F931F937C015B
:105AE0000E94682D8C01C7010E94DF2B9C01200FB2
:105AF000311FC9011F910F91FF90EF9008950895F4
:105B00001F920F920FB60F9211242F933F934F9332
:105B10008F939F93EF93FF938091C00082FD1DC0F0
:105B20004091C6002091F1053091F2052F5F3F4F63
:105B30002F7330708091F3059091F4052817390781
:105B400071F0E091F105F091F205EF54FA4F4083C6
:105B50003093F2052093F10502C08091C600FF91B9
:105B6000EF919F918F914F913F912F910F900FBE89
:105B70000F901F9018951F920F920FB60F9211243D
:105B80002F933F938F939F93EF93FF93209135062D
:105B900030913606809137069091380628173907DC
:105BA00031F48091C1008F7D8093C10014C0E091D9
:105BB0003706F0913806EB50FA4F20818091370676
:105BC0009091380601968F73907090933806809369
:105BD00037062093C600FF91EF919F918F913F91DF
:105BE0002F910F900FBE0F901F901895A0E0B0E07E
:105BF000ECEFFDE20C942C30FC011382128288EE53
:105C000093E0A0E0B0E084839583A683B7838BE81C
:105C100093E0918380837587648757874687318BAC
:105C2000208B138B028BF58AE48AD78AC68AB18EC1
:105C3000A08E938E828E8F85848F8889858F8989A7
:105C4000868F8A89878F8B8980A32096ECE00C94BD
:105C50004830AF92BF92DF92EF92FF920F931F9363
:105C6000CF93DF93EC017A018B01DD24403081EE8C
:105C7000580780E0680780E0780711F0DD24D394AE
:105C800091E0A92EB12CEC89FD89DD2069F0C501D8
:105C900008A002C0880F991F0A94E2F7808360E091
:105CA00079E08DE390E005C0108260E874E88EE151
:105CB00090E0A80197010E94E92F21503040404018
:105CC0005040569547953795279580E12030380705
:105CD00020F0DD2011F0DD24D6CFE889F98930836A
:105CE000EA89FB89208319A2EE89FF89408121E09E
:105CF00030E0C9010C8C02C0880F991F0A94E2F7AA
:105D0000482B4083EE89FF894081C9010D8C02C078
:105D1000880F991F0A94E2F7482B4083EE89FF8988
:105D20004081C9010E8C02C0880F991F0A94E2F7C6
:105D3000482B4083EE89FF8980810F8C02C0220F9F
:105D4000331F0A94E2F7209528232083DF91CF9117
:105D50001F910F91FF90EF90DF90BF90AF9008954B
:105D6000DC011C96ED91FC911D97E05CFF4F2191A9
:105D7000319180819181281B390B2F733070C901BB
:105D8000089589E396E00E94B02E892B11F00E94BD
:105D90007F2D0895DC011C96ED91FC911D97E05C30
:105DA000FF4F20813181E054F040DF01AE5BBF4FF7
:105DB0008D919C9111972817390719F42FEF3FEF18
:105DC00007C08D919C91E80FF91F8081282F30E04A
:105DD000C9010895DC011C96ED91FC911D97E05CD2
:105DE000FF4F20813181E054F040DF01AE5BBF4FB7
:105DF0008D919C9111972817390719F42FEF3FEFD8
:105E000010C08D919C911197E80FF91F20818D9101
:105E10009C91119701968F73907011969C938E931D
:105E200030E0C9010895DC0191968C919197882307
:105E300039F05496ED91FC915597808186FFF9CF0A
:105E400091961C920895CF93DF93EC01EE85FF8528
:105E5000E05CFF4F20813181E054F0402F5F3F4FE5
:105E60002F733070DF01AE5BBF4F8D919C91119706
:105E700028173907D1F3E05CFF4F80819181E0540E
:105E8000F040E80FF91F6083EE85FF85E05CFF4F6F
:105E900031832083EE89FF89208181E090E00F8C9F
:105EA00002C0880F991F0A94E2F7282B208381E013
:105EB00089A3EC89FD8980818064808381E090E002
:105EC000DF91CF9108958F929F92AF92BF92CF9220
:105ED000DF92EF92FF920F931F9300D000D00F92AA
:105EE000EDB7FEB7319684E0ADB7BEB711968C938F
:105EF00083E0818387E0828385E0838381E08483FC
:105F000089E396E061EB75E045EF55E025EC30E084
:105F100004EC10E0B0ECEB2EF12CA1ECCA2ED12C4D
:105F2000F2ECAF2EB12CE6EC8E2E912C0E94F62DC9
:105F30000F900F900F900F900F901F910F91FF9067
:105F4000EF90DF90CF90BF90AF909F908F9008958B
:105F5000CF93DF930E94662A0E941B28C1ECDEE2E9
:105F60000E940D122097E1F30E94C12EF9CF629F8B
:105F7000D001739FF001829FE00DF11D649FE00D41
:105F8000F11D929FF00D839FF00D749FF00D659FA2
:105F9000F00D9927729FB00DE11DF91F639FB00DA1
:105FA000E11DF91FBD01CF011124089597FB092EB2
:105FB00007260AD077FD04D086D006D000201AF438
:105FC000709561957F4F0895F6F7909581959F4F55
:105FD0000895A1E21A2EAA1BBB1BFD010DC0AA1F2A
:105FE000BB1FEE1FFF1FA217B307E407F50720F042
:105FF000A21BB30BE40BF50B661F771F881F991FBD
:106000001A9469F760957095809590959B01AC0105
:10601000BD01CF01089597FB092E05260ED057FD2F
:1060200004D0D7DF0AD0001C38F450954095309545
:1060300021953F4F4F4F5F4F0895F6F7909580950C
:10604000709561957F4F8F4F9F4F08952F923F928C
:106050004F925F926F927F928F929F92AF92BF9278
:10606000CF92DF92EF92FF920F931F93CF93DF9324
:10607000CDB7DEB7CA1BDB0B0FB6F894DEBF0FBE81
:10608000CDBF09942A88398848885F846E847D84CE
:106090008C849B84AA84B984C884DF80EE80FD80D0
:1060A0000C811B81AA81B981CE0FD11D0FB6F89446
:1060B000DEBF0FBECDBFED010895EE0FFF1F0590AF
:1060C000F491E02D0994AA1BBB1B51E107C0AA1F44
:1060D000BB1FA617B70710F0A61BB70B881F991F89
:1060E0005A95A9F780959095BC01CD01089591111D
:1060F00006C0803219F089508550D0F7089599274D
:0861000088270895F894FFCFF1
:106108004E6F005965730054582074696D656F753A
:106118007421006D6F64756C65206C6F636B6564CA
:106128003F00486F70206368616E6E656C200020C8
:1061380040200053004E2F4100386368002C002C8B
:10614800205B005D20280029004E4F5420454E4119
:10615800424C45440053656E64696E6720736574EC
:1061680074696E677320746F2052580A0052657301
:10617800657474696E672073657474696E677320DB
:106188006F6E2052580A0041626F72746564206510
:10619800646974730A00696E76616C69642073655A
:1061A8006C656374696F6E000D0A496E76616C697F
:1061B8006420696E707574202D2064697363617240
:1061C8006465642107007363616E6E6572206D6F8C
:1061D80064650053657474696E67732073617665CE
:1061E8006420746F20454550524F4D0A0052657621
:1061F80065727465642073657474696E677320666C
:10620800726F6D20454550524F4D0A004C6F6164C6
:10621800656420666163746F727920646566617570
:106228006C74730A004B657920616E642063686141
:106238006E6E656C732072616E646F6D697A6564E9
:106248000A004F70656E4C52536E67205458207385
:1062580074617274696E672000206F6E2048572041
:106268000050504D0052535349005344410053438A
:106278004C00525844005458440041494E004C4286
:106288004545500053504B54524D0053425553000E
:1062980053554D44004C4C494E440000342B3400B7
:1062A8003800382B340031320031322B340031368B
:1062B8000001000000C01200001A400AA1204EA5EB
:1062C800001B1E27522C23308025000005400AA100
:1062D800204EA50020244EA52C2330004B0000069C
:1062E800400AD0009D49007B289D492C233000E1BD
:1062F800000005400A4501D7DC03B81E0EBF002385
:106308002E48E801008A400A6001555502AD1E205A
:10631800000023C88025000005400AA1204EA500E2
:1063280020244EA52C2330000200020002000200A7
:106338000200020002000200020002000200020045
:1063480002000200020002FF01610265026A026E99
:1063580002720276027A027E0284028B0290029511
:10636800029B029B029B029B0235019C02A002A297
:1063780002A602A902AE02350100070B0C10111586
:1063880000160A1322312900000000232F922BB097
:086398002EEA2ECA2E132F007D
:107E00000F92CDB7DEB7112484B714BE81FFF1D035
:107E100082E08093C00088E18093C10086E0809377
:107E2000C20080E18093C4008EE0CDD088249924E4
:107E3000CC24C394F5E0DF2EE1E1EE2E73E0F72EC3
:107E4000B6D0082F813479F4B2D08983C2D0898129
:107E5000823811F481E005C0813811F485E001C059
:107E600083E09ED09AC0823411F484E103C085344B
:107E700019F485E0B6D091C0853561F498D0082F0B
:107E800010E095D090E0982E8824802A912A880CC2
:107E9000991C82C0863521F484E0A3D080E0E1CF34
:107EA000843609F04CC083D082D0A82E80D0B82E62
:107EB00000E011E07CD0F80181938F01AE16D1F77C
:107EC00088D0FB2DF53489F4E0E0F1E00BC0F9999E
:107ED000FECF92BC81BC0894811C911C819180BD15
:107EE000FA9AF99AEA1598F358C08B2D863409F05E
:107EF00054C0F401F7BEE89507B600FCFDCFF401CD
:107F0000A0E0B1E02C9130E011968C91119790E0B7
:107F1000982F8827822B932B12960C01C7BEE895C9
:107F20001124329681E0A038B80761F7F401D7BE7A
:107F3000E89507B600FCFDCFE7BEE8952EC0843774
:107F4000F1F435D034D0182F32D0B82E42D0FB2DDA
:107F5000F63421F4F40105914F010CC0FB2DF534EA
:107F600049F4F999FECF92BC81BC0894811C911C04
:107F7000F89A00B5802F14D0115049F70EC08537FC
:107F800039F427D08EE10CD085E90AD08FE069CF93
:107F9000813511F488E017D01CD080E101D050CF9A
:107FA0009091C00095FFFCCF8093C600089580910A
:107FB000C00087FFFCCF8091C00084FD01C0A89560
:107FC0008091C6000895E0E6F0E098E19083808318
:107FD0000895EDDF803219F088E0F5DFFFCF84E10E
:107FE000DFCF1F93182FE3DF1150E9F7F2DF1F9166
:0E7FF0000895282E80E0E7DFEE27FF27099492
:027FFE0001057B
:0400000300007E007B
:00000001FF
